
Getting Started with AVR Complete PWM Driver.elf:     file format elf32-avr

Sections:
Idx Name          Size      VMA       LMA       File off  Algn
  0 .text         00000476  00000000  00000000  00000074  2**1
                  CONTENTS, ALLOC, LOAD, READONLY, CODE
  1 .bss          00000002  00800060  00800060  000004ea  2**0
                  ALLOC
  2 .comment      00000030  00000000  00000000  000004ea  2**0
                  CONTENTS, READONLY
  3 .debug_aranges 00000068  00000000  00000000  0000051a  2**0
                  CONTENTS, READONLY, DEBUGGING
  4 .debug_info   0000022d  00000000  00000000  00000582  2**0
                  CONTENTS, READONLY, DEBUGGING
  5 .debug_abbrev 00000150  00000000  00000000  000007af  2**0
                  CONTENTS, READONLY, DEBUGGING
  6 .debug_line   00000190  00000000  00000000  000008ff  2**0
                  CONTENTS, READONLY, DEBUGGING
  7 .debug_frame  00000114  00000000  00000000  00000a90  2**2
                  CONTENTS, READONLY, DEBUGGING
  8 .debug_str    0000023a  00000000  00000000  00000ba4  2**0
                  CONTENTS, READONLY, DEBUGGING
  9 .debug_loc    000001c7  00000000  00000000  00000dde  2**0
                  CONTENTS, READONLY, DEBUGGING
 10 .debug_ranges 00000058  00000000  00000000  00000fa5  2**0
                  CONTENTS, READONLY, DEBUGGING

Disassembly of section .text:

00000000 <__vectors>:
   0:	0e c0       	rjmp	.+28     	; 0x1e <__ctors_end>
   2:	1d c0       	rjmp	.+58     	; 0x3e <__bad_interrupt>
   4:	1c c0       	rjmp	.+56     	; 0x3e <__bad_interrupt>
   6:	1c c0       	rjmp	.+56     	; 0x40 <__vector_3>
   8:	1a c0       	rjmp	.+52     	; 0x3e <__bad_interrupt>
   a:	19 c0       	rjmp	.+50     	; 0x3e <__bad_interrupt>
   c:	18 c0       	rjmp	.+48     	; 0x3e <__bad_interrupt>
   e:	17 c0       	rjmp	.+46     	; 0x3e <__bad_interrupt>
  10:	16 c0       	rjmp	.+44     	; 0x3e <__bad_interrupt>
  12:	21 c0       	rjmp	.+66     	; 0x56 <__vector_9>
  14:	52 c0       	rjmp	.+164    	; 0xba <__vector_10>
  16:	13 c0       	rjmp	.+38     	; 0x3e <__bad_interrupt>
  18:	12 c0       	rjmp	.+36     	; 0x3e <__bad_interrupt>
  1a:	11 c0       	rjmp	.+34     	; 0x3e <__bad_interrupt>
  1c:	10 c0       	rjmp	.+32     	; 0x3e <__bad_interrupt>

0000001e <__ctors_end>:
  1e:	11 24       	eor	r1, r1
  20:	1f be       	out	0x3f, r1	; 63
  22:	cf e5       	ldi	r28, 0x5F	; 95
  24:	d2 e0       	ldi	r29, 0x02	; 2
  26:	de bf       	out	0x3e, r29	; 62
  28:	cd bf       	out	0x3d, r28	; 61

0000002a <__do_clear_bss>:
  2a:	20 e0       	ldi	r18, 0x00	; 0
  2c:	a0 e6       	ldi	r26, 0x60	; 96
  2e:	b0 e0       	ldi	r27, 0x00	; 0
  30:	01 c0       	rjmp	.+2      	; 0x34 <.do_clear_bss_start>

00000032 <.do_clear_bss_loop>:
  32:	1d 92       	st	X+, r1

00000034 <.do_clear_bss_start>:
  34:	a2 36       	cpi	r26, 0x62	; 98
  36:	b2 07       	cpc	r27, r18
  38:	e1 f7       	brne	.-8      	; 0x32 <.do_clear_bss_loop>
  3a:	89 d0       	rcall	.+274    	; 0x14e <main>
  3c:	1a c2       	rjmp	.+1076   	; 0x472 <_exit>

0000003e <__bad_interrupt>:
  3e:	e0 cf       	rjmp	.-64     	; 0x0 <__vectors>

00000040 <__vector_3>:
void Timer_Frequency(int freq);
void PWM_Init(void);
void milliS_Timer(int milliS);

ISR(TIMER1_COMPA_vect)
{
  40:	1f 92       	push	r1
  42:	0f 92       	push	r0
  44:	0f b6       	in	r0, 0x3f	; 63
  46:	0f 92       	push	r0
  48:	11 24       	eor	r1, r1
	PORTB|=(1<<PORTB0);
  4a:	c0 9a       	sbi	0x18, 0	; 24
}
  4c:	0f 90       	pop	r0
  4e:	0f be       	out	0x3f, r0	; 63
  50:	0f 90       	pop	r0
  52:	1f 90       	pop	r1
  54:	18 95       	reti

00000056 <__vector_9>:
ISR(TIMER1_COMPB_vect)
{
  56:	1f 92       	push	r1
  58:	0f 92       	push	r0
  5a:	0f b6       	in	r0, 0x3f	; 63
  5c:	0f 92       	push	r0
  5e:	11 24       	eor	r1, r1
	PORTB&=~(1<<PORTB0);
  60:	c0 98       	cbi	0x18, 0	; 24
}
  62:	0f 90       	pop	r0
  64:	0f be       	out	0x3f, r0	; 63
  66:	0f 90       	pop	r0
  68:	1f 90       	pop	r1
  6a:	18 95       	reti

0000006c <PWM_BrightDim>:
	OCR1B = duty;	
}

void PWM_BrightDim(void)
{
	int Duty = OCR1B;
  6c:	8b b5       	in	r24, 0x2b	; 43
  6e:	90 e0       	ldi	r25, 0x00	; 0
	int Period = OCR1A;
  70:	4e b5       	in	r20, 0x2e	; 46
	static int direction;
	switch(direction)
  72:	20 91 60 00 	lds	r18, 0x0060
  76:	30 91 61 00 	lds	r19, 0x0061
  7a:	21 15       	cp	r18, r1
  7c:	31 05       	cpc	r19, r1
  7e:	21 f0       	breq	.+8      	; 0x88 <PWM_BrightDim+0x1c>
  80:	21 30       	cpi	r18, 0x01	; 1
  82:	31 05       	cpc	r19, r1
  84:	81 f0       	breq	.+32     	; 0xa6 <PWM_BrightDim+0x3a>
  86:	17 c0       	rjmp	.+46     	; 0xb6 <PWM_BrightDim+0x4a>
	{
		case UP:
			if(++Duty == (Period-1))	
  88:	01 96       	adiw	r24, 0x01	; 1
}

void PWM_BrightDim(void)
{
	int Duty = OCR1B;
	int Period = OCR1A;
  8a:	24 2f       	mov	r18, r20
  8c:	30 e0       	ldi	r19, 0x00	; 0
	static int direction;
	switch(direction)
	{
		case UP:
			if(++Duty == (Period-1))	
  8e:	21 50       	subi	r18, 0x01	; 1
  90:	31 09       	sbc	r19, r1
  92:	82 17       	cp	r24, r18
  94:	93 07       	cpc	r25, r19
  96:	79 f4       	brne	.+30     	; 0xb6 <PWM_BrightDim+0x4a>
				direction = DOWN;
  98:	21 e0       	ldi	r18, 0x01	; 1
  9a:	30 e0       	ldi	r19, 0x00	; 0
  9c:	30 93 61 00 	sts	0x0061, r19
  a0:	20 93 60 00 	sts	0x0060, r18
  a4:	08 c0       	rjmp	.+16     	; 0xb6 <PWM_BrightDim+0x4a>
			break;
		case DOWN:
			if(--Duty == 2)	
  a6:	01 97       	sbiw	r24, 0x01	; 1
  a8:	82 30       	cpi	r24, 0x02	; 2
  aa:	91 05       	cpc	r25, r1
  ac:	21 f4       	brne	.+8      	; 0xb6 <PWM_BrightDim+0x4a>
				direction = UP;
  ae:	10 92 61 00 	sts	0x0061, r1
  b2:	10 92 60 00 	sts	0x0060, r1
			break;
	}
	OCR1B = Duty;
  b6:	8b bd       	out	0x2b, r24	; 43
  b8:	08 95       	ret

000000ba <__vector_10>:
ISR(TIMER1_COMPB_vect)
{
	PORTB&=~(1<<PORTB0);
}
ISR(TIMER0_COMPA_vect)
{
  ba:	1f 92       	push	r1
  bc:	0f 92       	push	r0
  be:	0f b6       	in	r0, 0x3f	; 63
  c0:	0f 92       	push	r0
  c2:	11 24       	eor	r1, r1
  c4:	2f 93       	push	r18
  c6:	3f 93       	push	r19
  c8:	4f 93       	push	r20
  ca:	5f 93       	push	r21
  cc:	6f 93       	push	r22
  ce:	7f 93       	push	r23
  d0:	8f 93       	push	r24
  d2:	9f 93       	push	r25
  d4:	af 93       	push	r26
  d6:	bf 93       	push	r27
  d8:	ef 93       	push	r30
  da:	ff 93       	push	r31
	PWM_BrightDim();
  dc:	c7 df       	rcall	.-114    	; 0x6c <PWM_BrightDim>
}
  de:	ff 91       	pop	r31
  e0:	ef 91       	pop	r30
  e2:	bf 91       	pop	r27
  e4:	af 91       	pop	r26
  e6:	9f 91       	pop	r25
  e8:	8f 91       	pop	r24
  ea:	7f 91       	pop	r23
  ec:	6f 91       	pop	r22
  ee:	5f 91       	pop	r21
  f0:	4f 91       	pop	r20
  f2:	3f 91       	pop	r19
  f4:	2f 91       	pop	r18
  f6:	0f 90       	pop	r0
  f8:	0f be       	out	0x3f, r0	; 63
  fa:	0f 90       	pop	r0
  fc:	1f 90       	pop	r1
  fe:	18 95       	reti

00000100 <PWM_Init>:
	*/
}

void PWM_Init(void)
{
	TCCR1 |=(1<<CTC1)|(0 << CS13)|(0 << CS12)|(0 << CS11)|(1 << CS10);
 100:	80 b7       	in	r24, 0x30	; 48
 102:	81 68       	ori	r24, 0x81	; 129
 104:	80 bf       	out	0x30, r24	; 48
		Clock Select Bits 3, 2, 1, and 0
			The Clock Select bits 3, 2, 1, and 0 define the prescaling source of Timer/Counter1.
			When CS10 is 1, there'll be no prescaler.
		pg.89
	*/
	TIMSK |=(1 <<OCIE1A)|(1<<OCIE1B);
 106:	89 b7       	in	r24, 0x39	; 57
 108:	80 66       	ori	r24, 0x60	; 96
 10a:	89 bf       	out	0x39, r24	; 57
		Timer/Counter1 Output Compare Interrupt Enable
		Timer/Counter1 Overflow Interrupt Enable
		Reserved Bit
		pg92
	*/
	OCR1A = 50;// F_CPU/(10kHz*2*1)-1;
 10c:	82 e3       	ldi	r24, 0x32	; 50
 10e:	8e bd       	out	0x2e, r24	; 46
	OCR1B = 10;//Adjustable
 110:	8a e0       	ldi	r24, 0x0A	; 10
 112:	8b bd       	out	0x2b, r24	; 43
 114:	08 95       	ret

00000116 <milliS_Timer>:
		to the OCR1A value. 
	*/
}

void milliS_Timer(int milliS)
{
 116:	bc 01       	movw	r22, r24
	TCCR0A |=(1<<WGM01);
 118:	8a b5       	in	r24, 0x2a	; 42
 11a:	82 60       	ori	r24, 0x02	; 2
 11c:	8a bd       	out	0x2a, r24	; 42
			0 0 1 PWM, Phase Correct 0xFF TOP BOTTOM(2)
			0 1 0 CTC                OCRA Immediate MAX(1) (Selected)
			0 1 1 Fast PWM           0xFF BOTTOM(2) MAX(1)
		pg.79
	*/
	TCCR0B |=(1<CS02)|(0<<CS01)|(1<<CS00);
 11e:	83 b7       	in	r24, 0x33	; 51
 120:	81 60       	ori	r24, 0x01	; 1
 122:	83 bf       	out	0x33, r24	; 51
			 1    0    1   clk(I/O)/1024 (From prescaler) (Selected)
			 1    1    0   External clock source on T0 pin. Clock on falling edge.
			 1    1    1   External clock source on T0 pin. Clock on rising edge.
		pg.80
	*/
	TIMSK |= (1<<OCIE0A);
 124:	89 b7       	in	r24, 0x39	; 57
 126:	80 61       	ori	r24, 0x10	; 16
 128:	89 bf       	out	0x39, r24	; 57
		Timer/Counter0 Output Compare Match A Interrupt Enable
		Timer/Counter Output Compare Match B Interrupt Enable
		Timer/Counter0 Overflow Interrupt Enable
		Reserved Bits
	*/
	OCR0A = milliS*7.8125-1;
 12a:	88 27       	eor	r24, r24
 12c:	77 fd       	sbrc	r23, 7
 12e:	80 95       	com	r24
 130:	98 2f       	mov	r25, r24
 132:	a8 d0       	rcall	.+336    	; 0x284 <__floatsisf>
 134:	20 e0       	ldi	r18, 0x00	; 0
 136:	30 e0       	ldi	r19, 0x00	; 0
 138:	4a ef       	ldi	r20, 0xFA	; 250
 13a:	50 e4       	ldi	r21, 0x40	; 64
 13c:	2f d1       	rcall	.+606    	; 0x39c <__mulsf3>
 13e:	20 e0       	ldi	r18, 0x00	; 0
 140:	30 e0       	ldi	r19, 0x00	; 0
 142:	40 e8       	ldi	r20, 0x80	; 128
 144:	5f e3       	ldi	r21, 0x3F	; 63
 146:	0b d0       	rcall	.+22     	; 0x15e <__subsf3>
 148:	6f d0       	rcall	.+222    	; 0x228 <__fixunssfsi>
 14a:	69 bd       	out	0x29, r22	; 41
 14c:	08 95       	ret

0000014e <main>:
}

int main(void)
{
	DDRB |= (1 << DDB0);
 14e:	b8 9a       	sbi	0x17, 0	; 23
	DDRB &= ~(1 << DDB1);
 150:	b9 98       	cbi	0x17, 1	; 23
	sei();
 152:	78 94       	sei
	milliS_Timer(2);
 154:	82 e0       	ldi	r24, 0x02	; 2
 156:	90 e0       	ldi	r25, 0x00	; 0
 158:	de df       	rcall	.-68     	; 0x116 <milliS_Timer>
	PWM_Init();
 15a:	d2 df       	rcall	.-92     	; 0x100 <PWM_Init>
 15c:	ff cf       	rjmp	.-2      	; 0x15c <main+0xe>

0000015e <__subsf3>:
 15e:	50 58       	subi	r21, 0x80	; 128

00000160 <__addsf3>:
 160:	bb 27       	eor	r27, r27
 162:	aa 27       	eor	r26, r26
 164:	0e d0       	rcall	.+28     	; 0x182 <__addsf3x>
 166:	e0 c0       	rjmp	.+448    	; 0x328 <__fp_round>
 168:	d1 d0       	rcall	.+418    	; 0x30c <__fp_pscA>
 16a:	30 f0       	brcs	.+12     	; 0x178 <__addsf3+0x18>
 16c:	d6 d0       	rcall	.+428    	; 0x31a <__fp_pscB>
 16e:	20 f0       	brcs	.+8      	; 0x178 <__addsf3+0x18>
 170:	31 f4       	brne	.+12     	; 0x17e <__addsf3+0x1e>
 172:	9f 3f       	cpi	r25, 0xFF	; 255
 174:	11 f4       	brne	.+4      	; 0x17a <__addsf3+0x1a>
 176:	1e f4       	brtc	.+6      	; 0x17e <__addsf3+0x1e>
 178:	c6 c0       	rjmp	.+396    	; 0x306 <__fp_nan>
 17a:	0e f4       	brtc	.+2      	; 0x17e <__addsf3+0x1e>
 17c:	e0 95       	com	r30
 17e:	e7 fb       	bst	r30, 7
 180:	bc c0       	rjmp	.+376    	; 0x2fa <__fp_inf>

00000182 <__addsf3x>:
 182:	e9 2f       	mov	r30, r25
 184:	e2 d0       	rcall	.+452    	; 0x34a <__fp_split3>
 186:	80 f3       	brcs	.-32     	; 0x168 <__addsf3+0x8>
 188:	ba 17       	cp	r27, r26
 18a:	62 07       	cpc	r22, r18
 18c:	73 07       	cpc	r23, r19
 18e:	84 07       	cpc	r24, r20
 190:	95 07       	cpc	r25, r21
 192:	18 f0       	brcs	.+6      	; 0x19a <__addsf3x+0x18>
 194:	71 f4       	brne	.+28     	; 0x1b2 <__addsf3x+0x30>
 196:	9e f5       	brtc	.+102    	; 0x1fe <__addsf3x+0x7c>
 198:	fa c0       	rjmp	.+500    	; 0x38e <__fp_zero>
 19a:	0e f4       	brtc	.+2      	; 0x19e <__addsf3x+0x1c>
 19c:	e0 95       	com	r30
 19e:	0b 2e       	mov	r0, r27
 1a0:	ba 2f       	mov	r27, r26
 1a2:	a0 2d       	mov	r26, r0
 1a4:	0b 01       	movw	r0, r22
 1a6:	b9 01       	movw	r22, r18
 1a8:	90 01       	movw	r18, r0
 1aa:	0c 01       	movw	r0, r24
 1ac:	ca 01       	movw	r24, r20
 1ae:	a0 01       	movw	r20, r0
 1b0:	11 24       	eor	r1, r1
 1b2:	ff 27       	eor	r31, r31
 1b4:	59 1b       	sub	r21, r25
 1b6:	99 f0       	breq	.+38     	; 0x1de <__addsf3x+0x5c>
 1b8:	59 3f       	cpi	r21, 0xF9	; 249
 1ba:	50 f4       	brcc	.+20     	; 0x1d0 <__addsf3x+0x4e>
 1bc:	50 3e       	cpi	r21, 0xE0	; 224
 1be:	68 f1       	brcs	.+90     	; 0x21a <__addsf3x+0x98>
 1c0:	1a 16       	cp	r1, r26
 1c2:	f0 40       	sbci	r31, 0x00	; 0
 1c4:	a2 2f       	mov	r26, r18
 1c6:	23 2f       	mov	r18, r19
 1c8:	34 2f       	mov	r19, r20
 1ca:	44 27       	eor	r20, r20
 1cc:	58 5f       	subi	r21, 0xF8	; 248
 1ce:	f3 cf       	rjmp	.-26     	; 0x1b6 <__addsf3x+0x34>
 1d0:	46 95       	lsr	r20
 1d2:	37 95       	ror	r19
 1d4:	27 95       	ror	r18
 1d6:	a7 95       	ror	r26
 1d8:	f0 40       	sbci	r31, 0x00	; 0
 1da:	53 95       	inc	r21
 1dc:	c9 f7       	brne	.-14     	; 0x1d0 <__addsf3x+0x4e>
 1de:	7e f4       	brtc	.+30     	; 0x1fe <__addsf3x+0x7c>
 1e0:	1f 16       	cp	r1, r31
 1e2:	ba 0b       	sbc	r27, r26
 1e4:	62 0b       	sbc	r22, r18
 1e6:	73 0b       	sbc	r23, r19
 1e8:	84 0b       	sbc	r24, r20
 1ea:	ba f0       	brmi	.+46     	; 0x21a <__addsf3x+0x98>
 1ec:	91 50       	subi	r25, 0x01	; 1
 1ee:	a1 f0       	breq	.+40     	; 0x218 <__addsf3x+0x96>
 1f0:	ff 0f       	add	r31, r31
 1f2:	bb 1f       	adc	r27, r27
 1f4:	66 1f       	adc	r22, r22
 1f6:	77 1f       	adc	r23, r23
 1f8:	88 1f       	adc	r24, r24
 1fa:	c2 f7       	brpl	.-16     	; 0x1ec <__addsf3x+0x6a>
 1fc:	0e c0       	rjmp	.+28     	; 0x21a <__addsf3x+0x98>
 1fe:	ba 0f       	add	r27, r26
 200:	62 1f       	adc	r22, r18
 202:	73 1f       	adc	r23, r19
 204:	84 1f       	adc	r24, r20
 206:	48 f4       	brcc	.+18     	; 0x21a <__addsf3x+0x98>
 208:	87 95       	ror	r24
 20a:	77 95       	ror	r23
 20c:	67 95       	ror	r22
 20e:	b7 95       	ror	r27
 210:	f7 95       	ror	r31
 212:	9e 3f       	cpi	r25, 0xFE	; 254
 214:	08 f0       	brcs	.+2      	; 0x218 <__addsf3x+0x96>
 216:	b3 cf       	rjmp	.-154    	; 0x17e <__addsf3+0x1e>
 218:	93 95       	inc	r25
 21a:	88 0f       	add	r24, r24
 21c:	08 f0       	brcs	.+2      	; 0x220 <__addsf3x+0x9e>
 21e:	99 27       	eor	r25, r25
 220:	ee 0f       	add	r30, r30
 222:	97 95       	ror	r25
 224:	87 95       	ror	r24
 226:	08 95       	ret

00000228 <__fixunssfsi>:
 228:	98 d0       	rcall	.+304    	; 0x35a <__fp_splitA>
 22a:	88 f0       	brcs	.+34     	; 0x24e <__fixunssfsi+0x26>
 22c:	9f 57       	subi	r25, 0x7F	; 127
 22e:	90 f0       	brcs	.+36     	; 0x254 <__fixunssfsi+0x2c>
 230:	b9 2f       	mov	r27, r25
 232:	99 27       	eor	r25, r25
 234:	b7 51       	subi	r27, 0x17	; 23
 236:	a0 f0       	brcs	.+40     	; 0x260 <__stack+0x1>
 238:	d1 f0       	breq	.+52     	; 0x26e <__stack+0xf>
 23a:	66 0f       	add	r22, r22
 23c:	77 1f       	adc	r23, r23
 23e:	88 1f       	adc	r24, r24
 240:	99 1f       	adc	r25, r25
 242:	1a f0       	brmi	.+6      	; 0x24a <__fixunssfsi+0x22>
 244:	ba 95       	dec	r27
 246:	c9 f7       	brne	.-14     	; 0x23a <__fixunssfsi+0x12>
 248:	12 c0       	rjmp	.+36     	; 0x26e <__stack+0xf>
 24a:	b1 30       	cpi	r27, 0x01	; 1
 24c:	81 f0       	breq	.+32     	; 0x26e <__stack+0xf>
 24e:	9f d0       	rcall	.+318    	; 0x38e <__fp_zero>
 250:	b1 e0       	ldi	r27, 0x01	; 1
 252:	08 95       	ret
 254:	9c c0       	rjmp	.+312    	; 0x38e <__fp_zero>
 256:	67 2f       	mov	r22, r23
 258:	78 2f       	mov	r23, r24
 25a:	88 27       	eor	r24, r24
 25c:	b8 5f       	subi	r27, 0xF8	; 248
 25e:	39 f0       	breq	.+14     	; 0x26e <__stack+0xf>
 260:	b9 3f       	cpi	r27, 0xF9	; 249
 262:	cc f3       	brlt	.-14     	; 0x256 <__fixunssfsi+0x2e>
 264:	86 95       	lsr	r24
 266:	77 95       	ror	r23
 268:	67 95       	ror	r22
 26a:	b3 95       	inc	r27
 26c:	d9 f7       	brne	.-10     	; 0x264 <__stack+0x5>
 26e:	3e f4       	brtc	.+14     	; 0x27e <__stack+0x1f>
 270:	90 95       	com	r25
 272:	80 95       	com	r24
 274:	70 95       	com	r23
 276:	61 95       	neg	r22
 278:	7f 4f       	sbci	r23, 0xFF	; 255
 27a:	8f 4f       	sbci	r24, 0xFF	; 255
 27c:	9f 4f       	sbci	r25, 0xFF	; 255
 27e:	08 95       	ret

00000280 <__floatunsisf>:
 280:	e8 94       	clt
 282:	09 c0       	rjmp	.+18     	; 0x296 <__floatsisf+0x12>

00000284 <__floatsisf>:
 284:	97 fb       	bst	r25, 7
 286:	3e f4       	brtc	.+14     	; 0x296 <__floatsisf+0x12>
 288:	90 95       	com	r25
 28a:	80 95       	com	r24
 28c:	70 95       	com	r23
 28e:	61 95       	neg	r22
 290:	7f 4f       	sbci	r23, 0xFF	; 255
 292:	8f 4f       	sbci	r24, 0xFF	; 255
 294:	9f 4f       	sbci	r25, 0xFF	; 255
 296:	99 23       	and	r25, r25
 298:	a9 f0       	breq	.+42     	; 0x2c4 <__floatsisf+0x40>
 29a:	f9 2f       	mov	r31, r25
 29c:	96 e9       	ldi	r25, 0x96	; 150
 29e:	bb 27       	eor	r27, r27
 2a0:	93 95       	inc	r25
 2a2:	f6 95       	lsr	r31
 2a4:	87 95       	ror	r24
 2a6:	77 95       	ror	r23
 2a8:	67 95       	ror	r22
 2aa:	b7 95       	ror	r27
 2ac:	f1 11       	cpse	r31, r1
 2ae:	f8 cf       	rjmp	.-16     	; 0x2a0 <__floatsisf+0x1c>
 2b0:	fa f4       	brpl	.+62     	; 0x2f0 <__floatsisf+0x6c>
 2b2:	bb 0f       	add	r27, r27
 2b4:	11 f4       	brne	.+4      	; 0x2ba <__floatsisf+0x36>
 2b6:	60 ff       	sbrs	r22, 0
 2b8:	1b c0       	rjmp	.+54     	; 0x2f0 <__floatsisf+0x6c>
 2ba:	6f 5f       	subi	r22, 0xFF	; 255
 2bc:	7f 4f       	sbci	r23, 0xFF	; 255
 2be:	8f 4f       	sbci	r24, 0xFF	; 255
 2c0:	9f 4f       	sbci	r25, 0xFF	; 255
 2c2:	16 c0       	rjmp	.+44     	; 0x2f0 <__floatsisf+0x6c>
 2c4:	88 23       	and	r24, r24
 2c6:	11 f0       	breq	.+4      	; 0x2cc <__floatsisf+0x48>
 2c8:	96 e9       	ldi	r25, 0x96	; 150
 2ca:	11 c0       	rjmp	.+34     	; 0x2ee <__floatsisf+0x6a>
 2cc:	77 23       	and	r23, r23
 2ce:	21 f0       	breq	.+8      	; 0x2d8 <__floatsisf+0x54>
 2d0:	9e e8       	ldi	r25, 0x8E	; 142
 2d2:	87 2f       	mov	r24, r23
 2d4:	76 2f       	mov	r23, r22
 2d6:	05 c0       	rjmp	.+10     	; 0x2e2 <__floatsisf+0x5e>
 2d8:	66 23       	and	r22, r22
 2da:	71 f0       	breq	.+28     	; 0x2f8 <__floatsisf+0x74>
 2dc:	96 e8       	ldi	r25, 0x86	; 134
 2de:	86 2f       	mov	r24, r22
 2e0:	70 e0       	ldi	r23, 0x00	; 0
 2e2:	60 e0       	ldi	r22, 0x00	; 0
 2e4:	2a f0       	brmi	.+10     	; 0x2f0 <__floatsisf+0x6c>
 2e6:	9a 95       	dec	r25
 2e8:	66 0f       	add	r22, r22
 2ea:	77 1f       	adc	r23, r23
 2ec:	88 1f       	adc	r24, r24
 2ee:	da f7       	brpl	.-10     	; 0x2e6 <__floatsisf+0x62>
 2f0:	88 0f       	add	r24, r24
 2f2:	96 95       	lsr	r25
 2f4:	87 95       	ror	r24
 2f6:	97 f9       	bld	r25, 7
 2f8:	08 95       	ret

000002fa <__fp_inf>:
 2fa:	97 f9       	bld	r25, 7
 2fc:	9f 67       	ori	r25, 0x7F	; 127
 2fe:	80 e8       	ldi	r24, 0x80	; 128
 300:	70 e0       	ldi	r23, 0x00	; 0
 302:	60 e0       	ldi	r22, 0x00	; 0
 304:	08 95       	ret

00000306 <__fp_nan>:
 306:	9f ef       	ldi	r25, 0xFF	; 255
 308:	80 ec       	ldi	r24, 0xC0	; 192
 30a:	08 95       	ret

0000030c <__fp_pscA>:
 30c:	00 24       	eor	r0, r0
 30e:	0a 94       	dec	r0
 310:	16 16       	cp	r1, r22
 312:	17 06       	cpc	r1, r23
 314:	18 06       	cpc	r1, r24
 316:	09 06       	cpc	r0, r25
 318:	08 95       	ret

0000031a <__fp_pscB>:
 31a:	00 24       	eor	r0, r0
 31c:	0a 94       	dec	r0
 31e:	12 16       	cp	r1, r18
 320:	13 06       	cpc	r1, r19
 322:	14 06       	cpc	r1, r20
 324:	05 06       	cpc	r0, r21
 326:	08 95       	ret

00000328 <__fp_round>:
 328:	09 2e       	mov	r0, r25
 32a:	03 94       	inc	r0
 32c:	00 0c       	add	r0, r0
 32e:	11 f4       	brne	.+4      	; 0x334 <__fp_round+0xc>
 330:	88 23       	and	r24, r24
 332:	52 f0       	brmi	.+20     	; 0x348 <__fp_round+0x20>
 334:	bb 0f       	add	r27, r27
 336:	40 f4       	brcc	.+16     	; 0x348 <__fp_round+0x20>
 338:	bf 2b       	or	r27, r31
 33a:	11 f4       	brne	.+4      	; 0x340 <__fp_round+0x18>
 33c:	60 ff       	sbrs	r22, 0
 33e:	04 c0       	rjmp	.+8      	; 0x348 <__fp_round+0x20>
 340:	6f 5f       	subi	r22, 0xFF	; 255
 342:	7f 4f       	sbci	r23, 0xFF	; 255
 344:	8f 4f       	sbci	r24, 0xFF	; 255
 346:	9f 4f       	sbci	r25, 0xFF	; 255
 348:	08 95       	ret

0000034a <__fp_split3>:
 34a:	57 fd       	sbrc	r21, 7
 34c:	90 58       	subi	r25, 0x80	; 128
 34e:	44 0f       	add	r20, r20
 350:	55 1f       	adc	r21, r21
 352:	59 f0       	breq	.+22     	; 0x36a <__fp_splitA+0x10>
 354:	5f 3f       	cpi	r21, 0xFF	; 255
 356:	71 f0       	breq	.+28     	; 0x374 <__fp_splitA+0x1a>
 358:	47 95       	ror	r20

0000035a <__fp_splitA>:
 35a:	88 0f       	add	r24, r24
 35c:	97 fb       	bst	r25, 7
 35e:	99 1f       	adc	r25, r25
 360:	61 f0       	breq	.+24     	; 0x37a <__fp_splitA+0x20>
 362:	9f 3f       	cpi	r25, 0xFF	; 255
 364:	79 f0       	breq	.+30     	; 0x384 <__fp_splitA+0x2a>
 366:	87 95       	ror	r24
 368:	08 95       	ret
 36a:	12 16       	cp	r1, r18
 36c:	13 06       	cpc	r1, r19
 36e:	14 06       	cpc	r1, r20
 370:	55 1f       	adc	r21, r21
 372:	f2 cf       	rjmp	.-28     	; 0x358 <__fp_split3+0xe>
 374:	46 95       	lsr	r20
 376:	f1 df       	rcall	.-30     	; 0x35a <__fp_splitA>
 378:	08 c0       	rjmp	.+16     	; 0x38a <__fp_splitA+0x30>
 37a:	16 16       	cp	r1, r22
 37c:	17 06       	cpc	r1, r23
 37e:	18 06       	cpc	r1, r24
 380:	99 1f       	adc	r25, r25
 382:	f1 cf       	rjmp	.-30     	; 0x366 <__fp_splitA+0xc>
 384:	86 95       	lsr	r24
 386:	71 05       	cpc	r23, r1
 388:	61 05       	cpc	r22, r1
 38a:	08 94       	sec
 38c:	08 95       	ret

0000038e <__fp_zero>:
 38e:	e8 94       	clt

00000390 <__fp_szero>:
 390:	bb 27       	eor	r27, r27
 392:	66 27       	eor	r22, r22
 394:	77 27       	eor	r23, r23
 396:	cb 01       	movw	r24, r22
 398:	97 f9       	bld	r25, 7
 39a:	08 95       	ret

0000039c <__mulsf3>:
 39c:	0a d0       	rcall	.+20     	; 0x3b2 <__mulsf3x>
 39e:	c4 cf       	rjmp	.-120    	; 0x328 <__fp_round>
 3a0:	b5 df       	rcall	.-150    	; 0x30c <__fp_pscA>
 3a2:	28 f0       	brcs	.+10     	; 0x3ae <__mulsf3+0x12>
 3a4:	ba df       	rcall	.-140    	; 0x31a <__fp_pscB>
 3a6:	18 f0       	brcs	.+6      	; 0x3ae <__mulsf3+0x12>
 3a8:	95 23       	and	r25, r21
 3aa:	09 f0       	breq	.+2      	; 0x3ae <__mulsf3+0x12>
 3ac:	a6 cf       	rjmp	.-180    	; 0x2fa <__fp_inf>
 3ae:	ab cf       	rjmp	.-170    	; 0x306 <__fp_nan>
 3b0:	ef cf       	rjmp	.-34     	; 0x390 <__fp_szero>

000003b2 <__mulsf3x>:
 3b2:	cb df       	rcall	.-106    	; 0x34a <__fp_split3>
 3b4:	a8 f3       	brcs	.-22     	; 0x3a0 <__mulsf3+0x4>

000003b6 <__mulsf3_pse>:
 3b6:	99 23       	and	r25, r25
 3b8:	d9 f3       	breq	.-10     	; 0x3b0 <__mulsf3+0x14>
 3ba:	55 23       	and	r21, r21
 3bc:	c9 f3       	breq	.-14     	; 0x3b0 <__mulsf3+0x14>
 3be:	95 0f       	add	r25, r21
 3c0:	50 e0       	ldi	r21, 0x00	; 0
 3c2:	55 1f       	adc	r21, r21
 3c4:	aa 27       	eor	r26, r26
 3c6:	ee 27       	eor	r30, r30
 3c8:	ff 27       	eor	r31, r31
 3ca:	bb 27       	eor	r27, r27
 3cc:	00 24       	eor	r0, r0
 3ce:	08 94       	sec
 3d0:	67 95       	ror	r22
 3d2:	20 f4       	brcc	.+8      	; 0x3dc <__mulsf3_pse+0x26>
 3d4:	e2 0f       	add	r30, r18
 3d6:	f3 1f       	adc	r31, r19
 3d8:	b4 1f       	adc	r27, r20
 3da:	0a 1e       	adc	r0, r26
 3dc:	22 0f       	add	r18, r18
 3de:	33 1f       	adc	r19, r19
 3e0:	44 1f       	adc	r20, r20
 3e2:	aa 1f       	adc	r26, r26
 3e4:	66 95       	lsr	r22
 3e6:	a9 f7       	brne	.-22     	; 0x3d2 <__mulsf3_pse+0x1c>
 3e8:	77 95       	ror	r23
 3ea:	30 f4       	brcc	.+12     	; 0x3f8 <__mulsf3_pse+0x42>
 3ec:	f3 0f       	add	r31, r19
 3ee:	b4 1f       	adc	r27, r20
 3f0:	0a 1e       	adc	r0, r26
 3f2:	12 1e       	adc	r1, r18
 3f4:	08 f4       	brcc	.+2      	; 0x3f8 <__mulsf3_pse+0x42>
 3f6:	63 95       	inc	r22
 3f8:	33 0f       	add	r19, r19
 3fa:	44 1f       	adc	r20, r20
 3fc:	aa 1f       	adc	r26, r26
 3fe:	22 1f       	adc	r18, r18
 400:	76 95       	lsr	r23
 402:	99 f7       	brne	.-26     	; 0x3ea <__mulsf3_pse+0x34>
 404:	87 95       	ror	r24
 406:	20 f4       	brcc	.+8      	; 0x410 <__mulsf3_pse+0x5a>
 408:	b4 0f       	add	r27, r20
 40a:	0a 1e       	adc	r0, r26
 40c:	12 1e       	adc	r1, r18
 40e:	63 1f       	adc	r22, r19
 410:	44 0f       	add	r20, r20
 412:	aa 1f       	adc	r26, r26
 414:	22 1f       	adc	r18, r18
 416:	33 1f       	adc	r19, r19
 418:	86 95       	lsr	r24
 41a:	a9 f7       	brne	.-22     	; 0x406 <__mulsf3_pse+0x50>
 41c:	86 2f       	mov	r24, r22
 41e:	71 2d       	mov	r23, r1
 420:	60 2d       	mov	r22, r0
 422:	11 24       	eor	r1, r1
 424:	9f 57       	subi	r25, 0x7F	; 127
 426:	50 40       	sbci	r21, 0x00	; 0
 428:	8a f0       	brmi	.+34     	; 0x44c <__mulsf3_pse+0x96>
 42a:	e1 f0       	breq	.+56     	; 0x464 <__mulsf3_pse+0xae>
 42c:	88 23       	and	r24, r24
 42e:	4a f0       	brmi	.+18     	; 0x442 <__mulsf3_pse+0x8c>
 430:	ee 0f       	add	r30, r30
 432:	ff 1f       	adc	r31, r31
 434:	bb 1f       	adc	r27, r27
 436:	66 1f       	adc	r22, r22
 438:	77 1f       	adc	r23, r23
 43a:	88 1f       	adc	r24, r24
 43c:	91 50       	subi	r25, 0x01	; 1
 43e:	50 40       	sbci	r21, 0x00	; 0
 440:	a9 f7       	brne	.-22     	; 0x42c <__mulsf3_pse+0x76>
 442:	9e 3f       	cpi	r25, 0xFE	; 254
 444:	51 05       	cpc	r21, r1
 446:	70 f0       	brcs	.+28     	; 0x464 <__mulsf3_pse+0xae>
 448:	58 cf       	rjmp	.-336    	; 0x2fa <__fp_inf>
 44a:	a2 cf       	rjmp	.-188    	; 0x390 <__fp_szero>
 44c:	5f 3f       	cpi	r21, 0xFF	; 255
 44e:	ec f3       	brlt	.-6      	; 0x44a <__mulsf3_pse+0x94>
 450:	98 3e       	cpi	r25, 0xE8	; 232
 452:	dc f3       	brlt	.-10     	; 0x44a <__mulsf3_pse+0x94>
 454:	86 95       	lsr	r24
 456:	77 95       	ror	r23
 458:	67 95       	ror	r22
 45a:	b7 95       	ror	r27
 45c:	f7 95       	ror	r31
 45e:	e7 95       	ror	r30
 460:	9f 5f       	subi	r25, 0xFF	; 255
 462:	c1 f7       	brne	.-16     	; 0x454 <__mulsf3_pse+0x9e>
 464:	fe 2b       	or	r31, r30
 466:	88 0f       	add	r24, r24
 468:	91 1d       	adc	r25, r1
 46a:	96 95       	lsr	r25
 46c:	87 95       	ror	r24
 46e:	97 f9       	bld	r25, 7
 470:	08 95       	ret

00000472 <_exit>:
 472:	f8 94       	cli

00000474 <__stop_program>:
 474:	ff cf       	rjmp	.-2      	; 0x474 <__stop_program>
